:100000008B014F306200C828C32008300511BC2086
:100010000310061C0314A80CFF3E031D0628280825
:10002000C03A031D1828AB13AA01AD01AE01D128B7
:10003000AB1F2428CD3A031DD1284F30B0204B30C0
:10004000B0200D30B020D1282B1F2B281C3ADB30DC
:100050000319C030A8002B171B3A0319D1282B1302
:1000600028083F212A08EC3E031863282A0D8A013C
:1000700082072808AB00AB0D422800306028280812
:10008000AC006E28AB136E2800006E280000003014
:1000900060286E280000063060286E2800006E2858
:1000A00000002F30842830308428313084283230CA
:1000B0008428C0306028A8306028023060280230D0
:1000C0002806031DCF282B082A0203187028FF3AA0
:1000D000031D6E282D082E04031DCF28AA0AD1283F
:1000E000F23E031C8328031D7928980C980C981362
:1000F00018131802F13E031887282302F73E033E27
:10010000031C8728063E1A3E8400280880002A0A1D
:100110002C02031D6E282B08AC0231212D082E0461
:1001200003194B21CF282D08A3202E08A3288400D3
:100130009920000841219E20000844210008840ADB
:10014000A328A2200030C03A031DAA28DB30B0202B
:10015000DC30B0281B3A031DAF28AF200630DB3A55
:100160008515A90070300314BC20A90C031CC428F9
:10017000103E8511031DB3289B0026309A001B08F2
:100180009A0BC028000008008515103E0310B42803
:10019000860185010030650001306600A713AB01C0
:1001A000AB17051590308B00D4282710A710A60197
:1001B0002F21FA30AD00FE30AE004530B020A12036
:1001C0002608283EAC00A3203121A1204030B020D9
:1001D000A2208030B0200630B0209320C030A32071
:1001E000A830A3200230A3200230A3202F30972074
:1001F0001308240203180129920A0319910A03190A
:10020000900A9307AF30AD009330AE0031210E302D
:10021000840099200C3084009920143097201030ED
:1002200097205030B02027081339B02029084421E6
:10023000A2208030B020AA0126082A06031924290A
:10024000B7213F21AA0A1C299320A120AA01260830
:100250002A0603192F29B721A320AA0A2729C0306B
:10026000B0282C0844212F084121300844213108AE
:10027000412132084421C2304121B03044292A189A
:100280004429AD020130031CAE020130031CAD0253
:10029000031CAE0208000F08503A0E04031D0800AC
:1002A0001919A7131918A8299918AE29191E080099
:1002B0002508170226020319612926020319D828E6
:1002C00008001708A50013082406031DD8281808DD
:1002D0002C02A407A3070318A3171130271BAC296E
:1002E000A71A96292308F83E031CD5282008613C4C
:1002F00003198F29313CF63E031C832903309D00EE
:100300009E0168309329A10D2108A10DA10D21079F
:100310002207F03E2018643EA018C83E86009D01CA
:1003200001309E0080309F00A7169B299D0A260859
:100330009F02031C9E039E08031DA5291F087F3EE4
:100340000318A52927171F08A6298030A600D8283A
:10035000130AA400A50A1030A700D728130AA40086
:10036000A301A5019230A700D720A50A08008A01A1
:100370008A149D180A142A081D1880388200060E57
:10038000C22906080F39F63E0318073E3A3E080018
:1004000048345434543450342F3431342E3430344E
:1004100020343234303430340D340A340D340A345C
:100420003C347434693474346C3465343E34503440
:100430006F3472347434203442343C342F34743486
:10044000693474346C3465343E343C3462346F3413
:100450006434793420346F346E344C346F34613406
:1004600064343D34223466346F3472342834763444
:1004700061347234203469343D3430343B3469346F
:100480003C3437343B3469342B342B3429346434D2
:100490006F34633475346D3465346E3474342E3493
:1004A00066346F3472346D3473345B3430345D349D
:1004B0002E3465346C3465346D3465346E34743484
:1004C00073345B3469345D342E346334683465349A
:1004D00063346B34653464343D3430347834BF294C
:1004E000C1292634283432343C343C34693429342C
:1004F00022343E343C3466346F3472346D342034EC
:1005000061346334743469346F346E343D3461342F
:100510003E343C347334633472346934703474342C
:100520003E3466346F347234283476346134723435
:10053000203469343D3431343B3469343C3438340C
:100540003B3469342B342B34293464346F346334B2
:1005500075346D3465346E3474342E3477347234BB
:100560006934743465342834223442342E342234CD
:100570002B3469342B3422343C3449344E345034D7
:1005800055345434203454345934503445343D3483
:1005900063346834653463346B3462346F34783474
:1005A0003E343C34423452343E34223429343C34D8
:1005B0002F347334633472346934703474343E3499
:1005C0003C3469346E34703475347434203474348B
:1005D0007934703465343D347334753462346D3439
:1005E000693474342034763461346C347534653451
:1005F0003D3452346534613464343E343C346934BF
:100600006E34703475347434203474347934703406
:1006100065343D3462347534743474346F346E34FC
:100620002034763461346C34753465343D34573459
:10063000723469347434653420346F346E34433426
:100640006C34693463346B343D34223466346F3433
:1006500072342834763461347234203476343D3444
:100660003434303430342C3469343D3430343B3419
:1006700069343C3437343B3476342B343D34643481
:100680006F34633475346D3465346E3474342E34A1
:1006900066346F3472346D3473345B3430345D34AB
:1006A0002E3465346C3465346D3465346E34743492
:1006B00073345B3469345D342E34633468346534A8
:1006C00063346B34653464343C343C342B342B3425
:1006D000693429343B3474346F3470342E346C34C0
:1006E0006F3463346134743469346F346E342E344F
:1006F00068347234653466343D34763422343E34A2
:1007000048345434543450342F3431342E3430344B
:1007100020343234303430340D340A340D340A3459
:100720003C346134203468347234653466343D348A
:1007300061343E3450346F34723474344234203473
:1007400063346F346E34743472346F346C343C34CC
:100750002F3461343E343C34683472343E343C349B
:100760006134203468347234653466343D3468341E
:100770007434743470343A342F342F346B34793405
:100780006C346C3469346B346B3469342E346634B5
:100790006C347534663466342E346F347234673496
:1007A0002F34683461347234643477346134723491
:1007B00065342F343E347734773477347034693489
:1007C00063343234203468346F346D3465347034BB
:1007D0006134673465343C342F3461343E34203422
:1007E0000034003400340034003400340034003469
:1007F0000034003400340034003400340034003459
:02400E00FA3F77
:00000001FF
